:1000000000308A00AE2800000000F73065000519B6
:100010000B2800300C2801300038031D1128111462
:100020001116D1280E088E0A3C300E02031C262819
:100030008E010F088F0A3C300F02031C26288F0107
:100040001008900A1830100203189001D7281108E0
:100050004039003803197F28940114088900831659
:100060000814831208088C000C0A03197F2814084E
:100070008900831608148312080895000A301502B7
:10008000031C482820301502031848280630950222
:100090001A301502031C4E280C309502013014074B
:1000A0009700170889008316081483120808960021
:1000B0000A301602031C6228203016020318622838
:1000C000063096021A301602031C68280C3096027D
:1000D00015081002031D7C2816080F02031D7C283A
:1000E000023014079700170889008316081483123A
:1000F0000808FF3A03388600033094072D28D828D3
:10010000170803198B288928000000000000000050
:100110000000970B842898281308930A12081302EA
:10012000031D9C280030660006106430970080286C
:100130000030660006149301D928110801390038EF
:100140000319AD28133090008F018E011117DF3095
:100150009105FE30910503309200DA2884010430C5
:100160008C008C1DBB280730810181308400000881
:10017000C0390F3880006400813084000008C03925
:100180000C048000003066000610910101309200DE
:1001900093018101123090008F018E010B19D2283A
:1001A0000528CE280B110030660086171228272854
:0E01B0008C289D28003066008613CE28630040
:104200001900000004001900010008001900020054
:08421000040019000300000086
:08400000FF00FF00FF00FF00BC
:02400E00180098
:00000001FF
